 mouhid

 Timestamp is 4fb04cb8 (Mon May 14 12:07:20 2012)

 Preferred load address is 10000000

 Start         Length     Name                   Class
 0001:00000000 00000004H .CRT$XCA                CODE
 0001:00000004 00000004H .CRT$XCZ                CODE
 0001:00000008 00000004H .CRT$XIA                CODE
 0001:0000000c 00000004H .CRT$XIZ                CODE
 0001:00000010 00000004H .CRT$XPA                CODE
 0001:00000014 00000004H .CRT$XPZ                CODE
 0001:00000018 00000004H .CRT$XTA                CODE
 0001:0000001c 00000004H .CRT$XTZ                CODE
 0001:00000020 00000090H .rdata                  CODE
 0001:000000b0 00000023H .rdata$debug            CODE
 0001:000000d4 00000b14H .text                   CODE
 0001:00000be8 00000004H .xdata                  CODE
 0001:00000bec 00000028H .idata$2                CODE
 0001:00000c14 00000014H .idata$3                CODE
 0001:00000c28 00000064H .idata$4                CODE
 0001:00000c8c 000000aaH .idata$6                CODE
 0001:00000d40 0000006eH .edata                  CODE
 0002:00000000 00000064H .idata$5                DATA
 0002:00000064 00000008H .data                   DATA
 0002:0000006c 0000001cH .bss                    DATA
 0003:00000000 00000080H .pdata                  DATA

  Address         Publics by Value              Rva+Base       Lib:Object

 0000:00000000       ___safe_se_handler_table   00000000     <absolute>
 0000:00000000       ___safe_se_handler_count   00000000     <absolute>
 0001:00000000       __xc_a                     10001000     corelib0:crt0init.obj
 0001:00000004       __xc_z                     10001004     corelib0:crt0init.obj
 0001:00000008       __xi_a                     10001008     corelib0:crt0init.obj
 0001:0000000c       __xi_z                     1000100c     corelib0:crt0init.obj
 0001:00000010       __xp_a                     10001010     corelib0:crt0init.obj
 0001:00000014       __xp_z                     10001014     corelib0:crt0init.obj
 0001:00000018       __xt_a                     10001018     corelib0:crt0init.obj
 0001:0000001c       __xt_z                     1000101c     corelib0:crt0init.obj
 0001:0000005c       ??_C@_1CG@NNBNONKD@?$AAM?$AAo?$AAu?$AAs?$AAe?$AAA?$AAt?$AAt?$AAa?$AAc?$AAh?$AAe?$AAd?$AAE?$AAv?$AAe?$AAn?$AAt?$AA?$AA@ 1000105c     mouhid.obj
 0001:00000084       ??_C@_1CG@JHDABJCF@?$AAM?$AAo?$AAu?$AAs?$AAe?$AAD?$AAe?$AAt?$AAa?$AAc?$AAh?$AAe?$AAd?$AAE?$AAv?$AAe?$AAn?$AAt?$AA?$AA@ 10001084     mouhid.obj
 0001:000000d4       DllEntry                   100010d4 f   mouhid.obj
 0001:0000016c       HIDDeviceNotifications     1000116c f   mouhid.obj
 0001:000005c4       HIDDeviceAttach            100015c4 f   mouhid.obj
 0001:0000078c       HidP_GetSpecificValueCaps  1000178c f   hidparse:HIDPARSE.dll
 0001:0000079c       HidP_GetScaledUsageValue   1000179c f   hidparse:HIDPARSE.dll
 0001:000007ac       HidP_UsageListDifference   100017ac f   hidparse:HIDPARSE.dll
 0001:000007bc       HidP_GetUsages             100017bc f   hidparse:HIDPARSE.dll
 0001:000007cc       HidP_MaxUsageListLength    100017cc f   hidparse:HIDPARSE.dll
 0001:000007dc       HidP_GetCaps               100017dc f   hidparse:HIDPARSE.dll
 0001:000007ec       DriverMouseHookInitialize  100017ec f   MouHidStd:StandardMouse.obj
 0001:000007f4       DriverMouseHook            100017f4 f   MouHidStd:StandardMouse.obj
 0001:000007fc       EventModify                100017fc f   coredll:COREDLL.dll
 0001:0000080c       CloseHandle                1000180c f   coredll:COREDLL.dll
 0001:0000081c       CreateEventW               1000181c f   coredll:COREDLL.dll
 0001:0000082c       DisableThreadLibraryCalls  1000182c f   coredll:COREDLL.dll
 0001:0000083c       LocalAlloc                 1000183c f   coredll:COREDLL.dll
 0001:0000084c       mouse_event                1000184c f   coredll:COREDLL.dll
 0001:0000085c       LocalFree                  1000185c f   coredll:COREDLL.dll
 0001:0000086c       WaitForSingleObject        1000186c f   coredll:COREDLL.dll
 0001:0000087c       SetThreadPriority          1000187c f   coredll:COREDLL.dll
 0001:0000088c       CreateThread               1000188c f   coredll:COREDLL.dll
 0001:0000089c       _DllEntryCRTStartup        1000189c f   corelib0:pegdentry.obj
 0001:000008e4       __GSHandlerCheckCommon     100018e4 f   corelib0:gshandler.obj
 0001:00000920       __GSHandlerCheck           10001920 f   corelib0:gshandler.obj
 0001:00000944       __security_init_cookie     10001944 f   corelib0:seccinit.obj
 0001:000009a0       __security_check_cookie    100019a0 f   corelib0:armsecgs.obj
 0001:000009b4       __gsfailure                100019b4 f   corelib0:armsecgs.obj
 0001:00000af4       _cexit                     10001af4 f   corelib0:cexit.obj
 0001:00000b10       _initterm                  10001b10 f   corelib0:crt0dat.obj
 0001:00000b44       _cinit                     10001b44 f   corelib0:crt0dat.obj
 0001:00000b78       memcpy                     10001b78 f   corelib1:COREDLL.dll
 0001:00000b88       __security_gen_cookie2     10001b88 f   corelib1:COREDLL.dll
 0001:00000b98       __report_gsfailure         10001b98 f   corelib1:COREDLL.dll
 0001:00000ba8       free                       10001ba8 f   corelib1:COREDLL.dll
 0001:00000bb8       DeleteCriticalSection      10001bb8 f   coredll:COREDLL.dll
 0001:00000bc8       InterlockedExchange        10001bc8 f   coredll:COREDLL.dll
 0001:00000bd8       TerminateProcess           10001bd8 f   coredll:COREDLL.dll
 0001:00000bec       __IMPORT_DESCRIPTOR_HIDPARSE 10001bec     hidparse:HIDPARSE.dll
 0001:00000c00       __IMPORT_DESCRIPTOR_COREDLL 10001c00     coredll:COREDLL.dll
 0001:00000c14       __NULL_IMPORT_DESCRIPTOR   10001c14     hidparse:HIDPARSE.dll
 0002:00000000       __imp_CreateThread         10002000     coredll:COREDLL.dll
 0002:00000004       __imp_TerminateProcess     10002004     coredll:COREDLL.dll
 0002:00000008       __imp_InterlockedExchange  10002008     coredll:COREDLL.dll
 0002:0000000c       __imp_DeleteCriticalSection 1000200c     coredll:COREDLL.dll
 0002:00000010       __imp_EventModify          10002010     coredll:COREDLL.dll
 0002:00000014       __imp_CloseHandle          10002014     coredll:COREDLL.dll
 0002:00000018       __imp_CreateEventW         10002018     coredll:COREDLL.dll
 0002:0000001c       __imp_DisableThreadLibraryCalls 1000201c     coredll:COREDLL.dll
 0002:00000020       __imp_LocalAlloc           10002020     coredll:COREDLL.dll
 0002:00000024       __imp_mouse_event          10002024     coredll:COREDLL.dll
 0002:00000028       __imp_LocalFree            10002028     coredll:COREDLL.dll
 0002:0000002c       __imp_WaitForSingleObject  1000202c     coredll:COREDLL.dll
 0002:00000030       __imp_SetThreadPriority    10002030     coredll:COREDLL.dll
 0002:00000034       __imp_memcpy               10002034     corelib1:COREDLL.dll
 0002:00000038       __imp___security_gen_cookie2 10002038     corelib1:COREDLL.dll
 0002:0000003c       __imp___report_gsfailure   1000203c     corelib1:COREDLL.dll
 0002:00000040       __imp_free                 10002040     corelib1:COREDLL.dll
 0002:00000044       \177COREDLL_NULL_THUNK_DATA 10002044     coredll:COREDLL.dll
 0002:00000048       __imp_HidP_GetCaps         10002048     hidparse:HIDPARSE.dll
 0002:0000004c       __imp_HidP_MaxUsageListLength 1000204c     hidparse:HIDPARSE.dll
 0002:00000050       __imp_HidP_GetUsages       10002050     hidparse:HIDPARSE.dll
 0002:00000054       __imp_HidP_UsageListDifference 10002054     hidparse:HIDPARSE.dll
 0002:00000058       __imp_HidP_GetScaledUsageValue 10002058     hidparse:HIDPARSE.dll
 0002:0000005c       __imp_HidP_GetSpecificValueCaps 1000205c     hidparse:HIDPARSE.dll
 0002:00000060       \177HIDPARSE_NULL_THUNK_DATA 10002060     hidparse:HIDPARSE.dll
 0002:00000064       __security_cookie          10002064     corelib0:seccinit.obj
 0002:00000068       __security_cookie_complement 10002068     corelib0:seccinit.obj
 0002:00000078       _exitflag                  10002078     corelib0:cexit.obj
 0002:0000007c       __onexitend                1000207c     <common>
 0002:00000080       __onexitbegin              10002080     <common>
 0002:00000084       g_pcsExit                  10002084     <common>

 entry point at        0001:0000089c

 Static symbols

 0001:00000280       ?ProcessMouseReport@@YAXPAU_HID_MOUSE@@PADK@Z 10001280 f   mouhid.obj
 0001:00000500       ?MouseThreadProc@@YAKPAX@Z 10001500 f   mouhid.obj
 0001:000009f8       doexit                     100019f8 f   corelib0:cexit.obj
